:1000000090C2AAC2A9C2A8C2A7C2A6C2A5C2A4C2BF
:10001000A3C2A2C2A1C2A0C29FC29EC29DC29CC2D4
:100020009BC29AC299C200000000003E5B4F5B3E3B
:100030003E6B4F6B3E1C3E7C3E1C183C7E3C181CAD
:10004000577D571C1C5E7F5E1C00183C1800FFE7A4
:10005000C3E7FF0018241800FFE7DBE7FF30483A4A
:10006000060E2629792926407F050507407F0525AC
:100070003F5A3CE73C5A7F3E1C1C08081C1C3E7F34
:1000800014227F22145F5F005F5F06097F017F00FB
:100090006689956A606060606094A2FFA29408041B
:1000A0007E040810207E201008082A1C08081C2A3C
:1000B00008081E101010100C1E0C1E0C30383E3894
:1000C00030060E3E0E06000000000000005F00003B
:1000D0000007000700147F147F14242A7F2A1223AC
:1000E0001308646236495620500008070300001CBC
:1000F0002241000041221C002A1C7F1C2A08083EC5
:1001000008080080703000080808080800006060D7
:100110000020100804023E5149453E00427F400045
:1001200072494949462141494D331814127F10271D
:10013000454545393C4A494931412111090736496C
:10014000494936464949291E000014000000403440
:100150000000000814224114141414140041221445
:100160000802015909063E415D594E7C1211127C6C
:100170007F494949363E414141227F4141413E7FCD
:10018000494949417F090909013E414151737F08AD
:1001900008087F00417F41002040413F017F081453
:1001A00022417F404040407F021C027F7F040810B4
:1001B0007F3E4141413E7F090909063E4151215E92
:1001C0007F09192946264949493203017F01033F26
:1001D0004040403F1F2040201F3F4038403F6314B5
:1001E00008146303047804036159494D43007F41B7
:1001F00041410204081020004141417F04020102F4
:100200000440404040400003070800205454784018
:100210007F284444383844444428384444287F38AC
:100220005454541800087E090218A4A49C787F082E
:1002300004047800447D40002040403D007F1028A9
:10024000440000417F40007C047804787C0804046A
:10025000783844444438FC1824241818242418FC02
:100260007C08040408485454542404043F44243CA7
:100270004040207C1C2040201C3C4030403C442816
:100280001028444C9090907C4464544C44000836B0
:10029000410000007700000041360800020102041E
:1002A000023C2623263C1EA1A161123A4040207A3E
:1002B0003854545559215555794122545478422186
:1002C0005554784020545579400C1E5272123955BD
:1002D00055555939545454593955545458000045BA
:1002E0007C410002457D420001457C407D12111297
:1002F0007DF0282528F07C545545002054547C542A
:100300007C0A097F4932494949323A4444443A32E5
:100310004A4848303A4141217A3A42402078009D8B
:10032000A0A07D3D4242423D3D4040403D3C24FF37
:100330002424487E4943662B2FFC2F2BFF0929F6E6
:1003400020C0887E090320545479410000447D4137
:100350003048484A32384040227A007A0A0A727D90
:100360000D19317D2629292F2826292929263048AB
:100370004D4020380808080808080808382F10C819
:10038000ACBA2F102834FA00007B000008142A149D
:100390002222142A1408AA005500AAAA55AA55AA6E
:1003A000000000FF00101010FF00141414FF0010D4
:1003B00010FF00FF1010F010F0141414FC001414BF
:1003C000F700FF0000FF00FF1414F404FC141417DE
:1003D000101F10101F101F1414141F00101010F005
:1003E000000000001F101010101F10101010F0104F
:1003F000000000FF101010101010101010FF10005F
:100400000000FF140000FF00FF00001F1017000095
:10041000FC04F414141710171414F404F40000FF6F
:1004200000F714141414141414F700F71414141708
:100430001410101F101F141414F4141010F010F0E6
:1004400000001F101F0000001F14000000FC14001B
:1004500000F010F01010FF10FF141414FF1410100F
:10046000101F00000000F010FFFFFFFFFFF0F0F092
:10047000F0F0FFFFFF0000000000FFFF0F0F0F0F65
:100480000F3844443844FC4A4A4A347E0202060685
:10049000027E027E0263554941633844443C044075
:1004A0007E201E2006027E020299A5E7A5991C2A3D
:1004B000492A1C4C7201724C304A4D4D30304878FC
:1004C0004830BC625A463D3E494949007E0101011F
:1004D0007E2A2A2A2A2A44445F444440514A4440FE
:1004E00040444A51400000FF0103E080FF00000843
:1004F000086B6B083612362436060F090F0600000B
:1005000018180000001010003040FF0101001F010A
:10051000011E00191D1712003C3C3C3C000000006D
:10052000000011241FBECFE5D4E0DEBFCDBF10E038
:10053000A0E6B0E0E0EEF6E102C005900D92AE3923
:10054000B107D9F710E0AEE9B0E001C01D92A73BBA
:10055000B107E1F786D1C2C853CD82E022D6A0E030
:10056000B0E0BC01CD0181D72FE632E143E850E491
:100570000ED820E030E040E058E309D820E030E039
:1005800048EC52E404D845D7CB010895EF92FF928E
:100590000F931F9381E005D6A0E0B0E0BC01CD0130
:1005A00064D72FE632E143E850E4F1D720E030E0B1
:1005B00040E058E3ECD77B018C0123EC35EF40E2BF
:1005C00050E4E1D718161CF060E070E012C0C801DA
:1005D000B70123EC35EF40E250E44ED624EA30E791
:1005E0004DE35EE3AED620E030E048EC52E4CFD7F6
:1005F00010D7CB011F910F91FF90EF90089580E0ED
:10060000D0D5A0E0B0E0BC01CD012FD72FE632E17C
:1006100043E850E4BCD720E53BEE4FE151E4B7D7C7
:1006200020E030E040E058E3B2D720E030E048EC92
:1006300052E4ADD7EED6CB010895CF92DF92EF9280
:10064000FF920F931F93142F690190E070E071D413
:1006500080EDE82E87E0F82EC7010197F1F7812F92
:100660007AD4C7010197F1F7C60160E070E06AD45F
:10067000C7010197F1F7802F6AE010D8805D39D566
:10068000C7010197F1F7802F6AE008D8892F805DB4
:1006900030D5C7010197F1F71F910F91FF90EF90AF
:1006A000DF90CF900895BF92CF92DF92EF92FF92AA
:1006B0000F931F93B42E69013CD490EDE92E97E07F
:1006C000F92EC7010197F1F78B2D45D4C70101978A
:1006D000F1F7C60160E070E035D4C7010197F1F78A
:1006E000C80168EE73E0E6D7862F805D02D5C801A9
:1006F00068EE73E0DFD7182F092F64E670E0DAD7D1
:10070000862F805DF6D4812F902F64E670E0D2D7DB
:10071000182F092F8EE2EDD4C7010197F1F7812F31
:10072000902F6AE070E0C6D7862F805DE2D4812FDB
:10073000902F6AE070E0BED7805DDBD41F910F91EF
:10074000FF90EF90DF90CF90BF90089580E090E011
:1007500060E070E0EED383E0FED38FEF9FEF60E0C8
:1007600070E0F0D380E690E00AD585E0F4D380EE27
:1007700097E060E070E0E6D3CBD38091AA0090913F
:10078000AB0090939F0080939E008091B000909169
:10079000B1009093A1008093A00088E690E0EFD490
:1007A00083E0D9D38FEF9FEF60E070E0CBD381E798
:1007B00090E0E5D485E0CFD380EE97E060E070E094
:1007C000C1D3A6D38091AA009091AB009093A900C9
:1007D0008093A8008091B0009091B1009093A50003
:1007E0008093A40089E790E0CAD483E0B4D38FEF6C
:1007F0009FEF60E070E0A6D382E890E0C0D485E08F
:10080000AAD380EE97E060E070E09CD381D3809122
:10081000AA009091AB009093A7008093A6008091CE
:10082000B0009091B1009093A3008093A2008AE859
:1008300090E0A5D487EF5DD480E25BD483E08BD3D6
:100840008FEF9FEF60E070E07DD38DE890E097D46C
:1008500085EF90E06EEB70E06CD381E990E08FD48F
:100860000895AF92BF92CF92DF92FF920F931F93A2
:10087000CF93DF9301D1939880E090E0C3D180E1E2
:1008800097E228EC30E0F9013197F1F70197D9F7B9
:1008900083E011D380EA9FE00197F1F757DF88E802
:1008A00093E128EC30E0F9013197F1F70197D9F79E
:1008B000FF2430EDA32E37E0B32E20E2C22E2EE42B
:1008C000D22E9DDE8C01C5010197F1F76091A00049
:1008D0007091A10080919E0090919F0045E020EED4
:1008E00037E0E1DEC6010197F1F750DE8C01C5016A
:1008F0000197F1F76091A4007091A5008091A80084
:100900009091A90045E020EE37E0CDDEC6010197C9
:10091000F1F723DEEC01C5010197F1F78091A60004
:100920006091A20045E020EE37E00C2F86DEC60184
:100930000197F1F7C333D105A8F0FF2081F4939A12
:1009400083E009D380E098EF60E070E0FBD285EFB0
:1009500090E06EEB70E0EDD285E990E010D4FF24DA
:10096000F39416C0A897A0F481E0F81689F4939840
:1009700083E0F1D28FEF9FEF60E070E0E3D285EF8C
:1009800090E06EEB70E0D5D281E990E0F8D3FF24DF
:10099000C6010197F1F795CF8FEF81BB959A089526
:1009A00087B38C6287BB80E58DB9709A979A08955A
:1009B0008FB9779BFECF089592B39F7392BB9DE052
:1009C0009A95F1F78FB9779BFECF979A0895969AEB
:1009D00092E09A95F1F797988FB9779BFECF979A07
:1009E0000895BF92CF92DF92EF92FF920F931F93E1
:1009F000F82E192FB62EC72EE42E052FD22E8AE2FE
:100A0000DBDF812FE4DF8F2DE2DF802FE0DF8E2D13
:100A1000DEDF8BE2D1DF8C2DDADF8B2DD8DF8D2D61
:100A2000D6DF8D2DD4DF8CE2C7DF1F910F91FF90B1
:100A3000EF90DF90CF90BF900895959A80ED97E06A
:100A400028EC30E0F9013197F1F70197D9F7959843
:100A500080ED97E028EC30E0F9013197F1F701974C
:100A6000D9F7959A80ED97E028EC30E0F9013197BD
:100A7000F1F70197D9F708958FEF81BB959A90DF31
:100A8000DCDF81E099DF80E197E228EC30E0F901DA
:100A90003197F1F70197D9F78BEC8EDF89E397DF78
:100AA0008CE295DF80E093DF84E391DF82E08FDFEB
:100AB0008FEC82DF80E08BDF81EC89DF80E387DFF2
:100AC00088EE7ADF85E883DF80E081DF88E77FDFFB
:100AD0008AEE72DF80E07BDF80E079DF8DEE6CDF15
:100AE00084E675DF83E073DF82E171DF81E86FDF29
:100AF00087EF62DF80E26BDF80EC5EDF83E267DF3F
:100B000081EC5ADF80E163DF85EC56DF8EE35FDF47
:100B100088E25DDF87EC50DF86E859DF86E34CDF53
:100B200088E455DF8AE348DF85E551DF81EB44DF68
:100B300080E04DDF88E14BDF86EB3EDF88E047DF7A
:100B400082E845DF87E243DF82EF36DF80E03FDF88
:100B500086E232DF81E03BDF80EE2EDF8FE037DFA1
:100B600081E335DF8BE233DF8CE031DF8EE02FDF96
:100B700088E02DDF8EE42BDF81EF29DF87E327DF9D
:100B800087E025DF80E123DF83E021DF8EE01FDFC8
:100B900089E01DDF80E01BDF81EE0EDF80E017DFE4
:100BA0008EE015DF84E113DF83E011DF81E10FDFE9
:100BB00087E00DDF81E30BDF81EC09DF88E407DFED
:100BC00088E005DF8FE003DF8CE001DF81E3FFDEFB
:100BD00086E3FDDE8FE0FBDE81E1EEDE80EB94E07C
:100BE00028EC30E0F9013197F1F70197D9F789E264
:100BF000E3DE08951F93182F892FE9DE812FE7DEAA
:100C00001F910895EF92FF920F931F93CF93DF935D
:100C10007C014091990050919A0020919B00309165
:100C20009C00415050402150304080E090E060E016
:100C300070E0D7DE00E010E00CC0C701DBDF2196DA
:100C400080919B0090919C00C817D907B0F30F5F6B
:100C50001F4F8091990090919A000817190718F476
:100C6000C0E0D0E0EDCFDF91CF911F910F91FF90C9
:100C7000EF900895CF93DF93FC019B01EA018091EF
:100C8000990090919A00E817F90778F480919B00F9
:100C900090919C006817790740F4CF013196AF011D
:100CA0002F5F3F4F9EDECE01A5DFDF91CF910895EC
:100CB0000F931F93CF93DF93DC01EA0189018091A9
:100CC000990090919A00A817B90728F580919B0088
:100CD00090919C0068177907F0F4FB0131972091FF
:100CE0009B0030919C00CF01840F951F82179307C2
:100CF00030F0C0919B00D0919C00C61BD70BEC0F2D
:100D0000FD1FCD01AD019F016CDE03C0C80172DF84
:100D100021972097D9F7DF91CF911F910F910895D7
:100D20000F931F93CF93DF93FC01DB01EA0189014D
:100D30008091990090919A00E817F90730F5809119
:100D40009B0090919C0068177907F8F4AF0141501F
:100D500050402091990030919A00CA018C0F9D1F3C
:100D60008217930730F0C0919900D0919A00CE1B62
:100D7000DF0B4C0F5D1FCF01BD019D0132DE03C0B3
:100D8000C80138DF21972097D9F7DF91CF911F91C4
:100D90000F9108958F929F92AF92BF92CF92DF9260
:100DA000EF92FF920F931F937C016B015A0149014F
:100DB0009801B6DFB60161507040680D791DC7011A
:100DC000A5019801ADDFC701B601A401980170DF4C
:100DD0000894E108F108C7018A0D9B1DB601A40122
:100DE000980166DF1F910F91FF90EF90DF90CF90F9
:100DF000BF90AF909F908F900895CF92DF92EF9227
:100E0000FF920F931F93CF93DF93DC017A01E901E7
:100E100068018091990090919A00A817B90708F08D
:100E200041C080919B0090919C0068177907D0F594
:100E3000AD01415050402091990030919A00CA0173
:100E40008E0D9F1D8217930730F0E0909900F0906F
:100E50009A00EA1AFB0AFB01319720919B0030911E
:100E60009C00CF018C0F9D1F8217930730F0C0911B
:100E70009B00D0919C00C61BD70B4E0D5F1DEC0F45
:100E8000FD1FCD019F01ADDD8E0107C0C601B2DEA1
:100E900021972097D9F7015010400115110511F045
:100EA000E701F7CFDF91CF911F910F91FF90EF9066
:100EB000DF90CF9008951F93182F86E37DDD137088
:100EC000113049F0113028F0123039F01330F1F4BC
:100ED0000FC088E403C088E20CC088E878DD80EFAA
:100EE00090E090939A008093990080E491E00AC08A
:100EF00088EE6DDD80E491E090939A0080939900F4
:100F000080EF90E090939C0080939B001F91089548
:100F10008091B4009091B5009093AB008093AA00AB
:100F20008091AE009091AF009093B1008093B0009B
:100F300008959093B5008093B4007093AF006093D0
:100F4000AE0008959093B3008093B2007093AD000B
:100F50006093AC000895893028F4882309F481E077
:100F60008093B60008952F923F924F925F926F92B6
:100F70007F928F929F92AF92BF92CF92DF92EF9229
:100F8000FF920F931F93DF93CF93CDB7DEB72897D0
:100F90000FB6F894DEBF0FBECDBF1B013C832B8381
:100FA0001E830D835E2C98878F838091990090918A
:100FB0009A002F8138852817390708F081C0809161
:100FC0009B0090919C006817790708F079C06E2CFF
:100FD0007724C301880F991F860D971D880F991FCD
:100FE000820F931F181619060CF06AC0C30153E054
:100FF000880F991F5A95E1F7820D931D181619064F
:101000000CF05EC085E0489F5001112486E290E01C
:10101000A80EB91E49011A829A81953011F4442410
:1010200002C0F501449061017101198240FE12C0B5
:10103000F1E05F1631F48F819885B7014B815C81B7
:1010400017C0C401B601452D50E0252D30E00B81BD
:101050001C8118C02D813E818B819C812817390706
:1010600091F091E0591631F48F819885B701A9016B
:1010700001DE09C0C401B601452D50E0252D30E048
:101080000D811E81BADEE981EF5FE983C60CD71CB2
:101090000894E11CF11CE83011F04694C7CFFA81A6
:1010A000FF5FFA83860C971C2F8138852F5F3F4F97
:1010B00038872F830894A11CB11CF63009F0ACCFFF
:1010C00028960FB6F894DEBF0FBECDBFCF91DF914B
:1010D0001F910F91FF90EF90DF90CF90BF90AF9056
:1010E0009F908F907F906F905F904F903F902F9048
:1010F0000895EF920F931F93482F8A30B9F42091EF
:10110000AE003091AF008091B60090E0E3E0880F30
:10111000991FEA95E1F7820F931F9093AF00809398
:10112000AE001092B5001092B40025C08D3019F1B8
:101130008091B4009091B5006091AE007091AF00C5
:101140002091B2003091B3000091AC001091AD003D
:10115000E090B60008DF4091B4005091B500809156
:10116000B60026E0829FC0011124840F951F909342
:10117000B5008093B4001F910F91EF9008951F93D5
:10118000CF93DF93EC0110E002C0B3DF1F5FFE01DD
:10119000E10FF11D80818823C1F7DF91CF911F916D
:1011A00008950F931F93813049F0813028F08230E9
:1011B00039F0833041F406C013EC05C013ED03C0D1
:1011C00013EE01C013EF37D03CD080E943D081E06B
:1011D00041D0812F3FD083E03DD039D010E009C00D
:1011E00030D081E937D081E03CD0182F80E039D071
:1011F0002ED017FFF5CF25D080E92CD080E02AD063
:1012000026D01FD081E926D081E02BD0082F80E0A6
:1012100028D0182F1CD0902F80E0212F30E0282BD1
:10122000392B80E82130380710F020E030E0C90188
:101230001F910F91089511B887E480B984E086BFAB
:10124000089584EA86BF06B607FEFDCF089584E9B7
:1012500086BF089583B984E886BF06B607FEFDCF32
:1012600008958295880F880F807C846886BF06B6B3
:1012700007FEFDCF83B108955058BB27AA270ED093
:1012800048C139D130F03ED120F031F49F3F11F404
:101290001EF42EC10EF4E095E7FB24C1E92F4AD1DC
:1012A00080F3BA17620773078407950718F071F483
:1012B0009EF562C10EF4E0950B2EBA2FA02D0B0106
:1012C000B90190010C01CA01A0011124FF27591B8B
:1012D00099F0593F50F4503E68F11A16F040A22F91
:1012E000232F342F4427585FF3CF46953795279502
:1012F000A795F0405395C9F77EF41F16BA0B620B01
:10130000730B840BBAF09150A1F0FF0FBB1F661F47
:10131000771F881FC2F70EC0BA0F621F731F841F8A
:1013200048F4879577956795B795F7959E3F08F0B0
:10133000B3CF9395880F08F09927EE0F979587956F
:1013400008950CD0E6C0DED040F0D5D030F021F4C6
:101350005F3F19F0C7C0511110C1CAC0EBD098F35C
:101360009923C9F35523B1F3951B550BBB27AA2726
:1013700062177307840738F09F5F5F4F220F331F98
:10138000441FAA1FA9F333D00E2E3AF0E0E830D064
:1013900091505040E695001CCAF729D0FE2F27D067
:1013A000660F771F881FBB1F261737074807AB0735
:1013B000B0E809F0BB0B802DBF01FF2793585F4FAA
:1013C0002AF09E3F510568F08DC0D7C05F3FECF317
:1013D000983EDCF3869577956795B795F7959F5F6F
:1013E000C9F7880F911D9695879597F90895E1E0C3
:1013F000660F771F881FBB1F621773078407BA0722
:1014000020F0621B730B840BBA0BEE1F88F7E0957C
:10141000089598D088F09F5790F0B92F9927B75129
:10142000A0F0D1F0660F771F881F991F1AF0BA95A8
:10143000C9F712C0B13081F09FD0B1E008959CC0CF
:10144000672F782F8827B85F39F0B93FCCF386959E
:1014500077956795B395D9F73EF4909580957095FB
:1014600061957F4F8F4F9F4F0895E89409C097FB78
:101470003EF490958095709561957F4F8F4F9F4F6B
:101480009923A9F0F92F96E9BB279395F6958795AF
:1014900077956795B795F111F8CFFAF4BB0F11F472
:1014A00060FF1BC06F5F7F4F8F4F9F4F16C0882319
:1014B00011F096E911C0772321F09EE8872F762F4F
:1014C00005C0662371F096E8862F70E060E02AF090
:1014D0009A95660F771F881FDAF7880F969587957C
:1014E00097F9089597F99F6780E870E060E00895A4
:1014F0009FEF80EC089500240A941616170618062C
:101500000906089500240A94121613061406050607
:101510000895092E0394000C11F4882352F0BB0F98
:1015200040F4BF2B11F460FF04C06F5F7F4F8F4FFB
:101530009F4F089557FD9058440F551F59F05F3F36
:1015400071F04795880F97FB991F61F09F3F79F0E5
:1015500087950895121613061406551FF2CF469567
:10156000F1DF08C0161617061806991FF1CF8695E9
:101570007105610508940895E894BB2766277727CD
:10158000CB0197F9089566D008F48FEF08950BD03A
:10159000C0CFB1DF28F0B6DF18F0952309F0A2CF55
:1015A000A7CF1124EACFC6DFA0F3959FD1F3950F03
:1015B00050E0551F629FF001729FBB27F00DB11DD7
:1015C000639FAA27F00DB11DAA1F649F6627B00D67
:1015D000A11D661F829F2227B00DA11D621F739F50
:1015E000B00DA11D621F839FA00D611D221F749F5E
:1015F0003327A00D611D231F849F600D211D822FA5
:10160000762F6A2F11249F5750408AF0E1F08823EB
:101610004AF0EE0FFF1FBB1F661F771F881F9150F8
:101620005040A9F79E3F510570F05CCFA6CF5F3FB9
:10163000ECF3983EDCF3869577956795B795F7952B
:10164000E7959F5FC1F7FE2B880F911D96958795B3
:1016500097F90895990F0008550FAA0BE0E8FEEFDF
:1016600016161706E807F907C0F012161306E40766
:10167000F50798F0621B730B840B950B39F40A265F
:1016800061F0232B242B252B21F408950A2609F43D
:10169000A140A6958FEF811D811D0895991B79E0CA
:1016A00004C0991F961708F0961B881F7A95C9F7F2
:1016B00080950895AA1BBB1B51E107C0AA1FBB1F41
:1016C000A617B70710F0A61BB70B881F991F5A95CE
:1016D000A9F780959095BC01CD010895F894FFCFAE
:1016E000564F4C54202D200030302E3030560A0AF0
:1016F00000414D50202D20200030302E3030410A46
:101700000A0054454D50202D200030300046414EF7
:0E171000004F4646004F4E20004001F0000002
:00000001FF
